:100000000C941E060C940E280C943B280C94460667
:100010000C9446060C9446060C9446060C94460630
:100020000C9446060C9446060C9425130C94460634
:100030000C9446060C9446060C9446060C94460610
:100040000C9468280C9446060C94562C0C94992C0D
:100050000C9446060C9446060C9446060C944606F0
:100060000C9446060C9446068918EB18CA18CD184D
:10007000D018D318D618D918DC18EB18E5181D1AA3
:100080001F1A1F1A1D1A1F1A1F1A1F1A1F1A1F1AAA
:100090001F1A1F1A1F1A1F1A1F1A1F1A1F1A1F1A98
:1000A000A3191F1A1F1A1F1A1F1A1F1A14191F1A11
:1000B0001F1A1F1A1F1A1F1A1F1A1F1A1F1A1F1A78
:1000C0001F1A1F1A1F1A1F1A1F1A1F1AAF19AF194A
:1000D000AF19AF19AF19AF19AF19AF19AF191F1A6F
:1000E0001F1A1F1A1F1A1F1A1F1A1419AE19AE1938
:1000F000AE19AE191F1ABC19C219C819CE19D419D4
:10010000DA19E019E619F019FA19041A0E1A551934
:1001100017191F1A1F1A1F1A1F1AA3191F1A1F1A9D
:100120001F1A1F1A1F1A1F1A1F1A1F1AAD19AD19ED
:10013000AD19AD191F1ABC19C219C819CE19D41995
:10014000DA19E019E619F019FA19041A0E1A5519F4
:1001500017191F1A1F1A1F1A1F1AA319521A521AF7
:10016000521A521A521A521A521A521A521A521A2F
:10017000521A521A521A691B691B691B691B691BA7
:10018000691B971AA11AAB1AB51A131B1D1B2C1B3E
:100190003D1BC51CDA1CE61CEF1CFE1C231D2C1D80
:1001A000751D3E1D87208D2093209A20A820CA20EF
:1001B000E820456E746572206D656E752E2E2E00DA
:1001C000546F67676C6564206D6963726F50504D42
:1001D00000546F67676C656420696E76657274653C
:1001E000642050504D2100546F67676C6564205443
:1001F00058206D7574696E672100546F67676C6570
:10020000642074656C656D65747279210050726F3D
:10021000746F636F6C206572726F72207769746897
:100220002052580054696D656F7574207768656E4B
:1002300020636F6E6E656374696E6720746F205201
:100240005800507265737320616E79206B65792058
:10025000746F2063616E63656C00436F6E6E6563DF
:1002600074696E6720746F2052582C20706F776508
:100270007220757020746865205258202877697440
:10028000682062696E6420706C7567206966206EF4
:100290006F74207573696E6720616C776179732064
:1002A00062696E642900546F67676C656420276912
:1002B0006D6D656469617465206F75747075742700
:1002C00000546F67676C65642027736C61766520E6
:1002D0006D6F64652700546F67676C6564202761E4
:1002E0006C776179732062696E642700546F676769
:1002F0006C65642050504D206368616E6E656C20A3
:100300006C696D69740053657420525353492069B8
:100310006E6A656374696F6E206368616E6E656C8A
:100320002028303D3D64697361626C652900536526
:10033000742050504D206D696E696D756D20737914
:100340006E630053657420626561636F6E20696E31
:1003500074657276616C0053657420626561636FC9
:100360006E2064656C617900536574206265616319
:100370006F6E206672657175656E637920696E2097
:10038000487A3A20303D64697361626C652C205074
:10039000783D504D52206368616E6E656C20782CFC
:1003A0002046783D465253206368616E6E656C202E
:1003B00078005365742050574D2073746F7020641B
:1003C000656C61792028302064697361626C6564B2
:1003D0002C20312D323535203D3D20302E317320FB
:1003E0002D2035306D696E29005365742050504DB5
:1003F0002073746F702064656C61792028302064EC
:10040000697361626C65642C20312D323535203D75
:100410003D20302E3173202D2035306D696E29003E
:10042000536574206661696C736166652064656CF0
:1004300061792028302064697361626C65642C20C6
:10044000312D323535203D3D20302E3173202D2089
:1004500035306D696E29002A2A2A2A2A2A2A2A2A50
:100460002A2A2A2A2A2A2A2A2A2A2A2A2A2A2A2AEC
:100470002A2A2A2A0052582041636B6564202D20C5
:1004800072657665727420737563636573736675E0
:100490006C21002A2A2A2A2A2A2A2A2A2A2A2A2AAD
:1004A0002A2A2A2A2A2A2A2A2A2A2A2A2A2A2A2AAC
:1004B000002A2A2A2A2A2A2A2A2A2A2A2A2A2A2AC6
:1004C0002A2A2A2A2A2A2A2A2A2A2A2A2A2A00528E
:1004D000582041636B6564202D20757064617465DC
:1004E000207375636365737366756C21002A2A2A0D
:1004F0002A2A2A2A2A2A2A2A2A2A2A2A2A2A2A2A5C
:100500002A2A2A2A2A2A2A2A2A2A0056616C696457
:100510002063686F69636573206172653A205B319F
:100520005D2D5B31365D20286368616E6E656C20E1
:10053000312D31362900536574206F7574707574D0
:1005400020666F7220706F727420005B585D2061AE
:10055000626F7274206368616E67657320616E6498
:10056000206578697420525820636F6E6669670051
:100570005B535D20736176652073657474696E6783
:100580007320746F205258005B525D20726576654F
:1005900072742052582073657474696E6773207486
:1005A0006F2064656661756C747300557365206EA9
:1005B000756D62657273205B312D445D20746F2010
:1005C0006564697420706F727473205B452D515D92
:1005D00020666F722073657474696E677300202DD6
:1005E00020726563656976657220636F6E66696700
:1005F000757261746F722C20727820737720000AF4
:100600000A6F70656E4C52536E67200053657420FC
:1006100073657269616C2062617564726174653AB8
:10062000200056616C69642063686F696365733A82
:100630002031202D20342B34202F2032202D203823
:10064000202F2033202D20382B34202F2034202D14
:10065000203132202F2035202D2031322B34202FF5
:100660002036202D20313600536574204368616E9A
:100670006E656C20636F6E6669673A20005365741F
:100680002044617461726174652028302D32293AEA
:10069000200053657420486F70206368616E6E653A
:1006A0006C7320286D61782032342C207365706162
:1006B000726174656420627920636F6D6D61732966
:1006C0002076616C69642076616C75657320312DCC
:1006D0003235353A2000536574206368616E6E656B
:1006E0006C2073706163696E6720287831306B48C5
:1006F0007A293A200053657420524620706F77653E
:10070000722028302D37293A200053657420524634
:10071000206D6167696320286865782920652E67E8
:100720002E20307844454144463030443A2000532E
:1007300065742062617365206672657175656E63AC
:10074000792028696E20487A293A20005B5A5D207A
:10075000656E746572207265636569766572206383
:100760006F6E66696775726174696F6E2075746902
:100770006C79005B465D20646973706C61792061FF
:10078000637475616C206672657175656E63696509
:10079000732075736564005B525D2063616C6375E3
:1007A0006C6174652072616E646F6D206B65792079
:1007B000616E6420686F70206C697374005B495DC2
:1007C000207265696E697469616C697A6520736508
:1007D0007474696E677320746F20736B65746368DB
:1007E0002064656661756C7473005B585D2072658A
:1007F00076657274206368616E67657320616E64EC
:100800002065786974206D656E75005B535D20739B
:100810006176652073657474696E677320746F20E8
:10082000454550524F4D20616E64206578697420B3
:100830006D656E7500557365206E756D62657273BA
:10084000205B302D395D20746F20656469742070E1
:100850006172616D657465727300202D2053797328
:1008600074656D20636F6E66696775726174696F18
:100870006E000A0A6F70656E4C52536E672000510D
:1008800029204F7574707574206265666F726520DB
:100890006C696E6B20283D465329203A2000502970
:1008A00020536C617665206D6F64652028657870D3
:1008B0006572696D656E74616C293A20004F29205C
:1008C00054696D65642042494E44206174207374FC
:1008D000617274757020203A20004E292050504DCE
:1008E000206F7574707574206C696D69746564200F
:1008F000202020203A200044495341424C454400E6
:100900004D292050504D205253534920746F20637D
:1009100068616E6E656C202020203A20004C2920F2
:1009200050504D206D696E696D756D2073796E63E1
:10093000202875732920203A200044495341424C15
:100940004544004B29204661696C736166652062ED
:100950006561636F6E20696E74762E2028312D32AA
:10096000353573293A20004A29204661696C736144
:10097000666520626561636F6E2064656C617920D5
:1009800028302D323535203D3E20313073202D204A
:100990003135306D696E293A200049292046616958
:1009A0006C7361666520626561636F6E206672714B
:1009B0002E203A200048292050574D2073746F7024
:1009C0002064656C6179202020202020203A2000BE
:1009D00047292050504D2073746F702064656C61FE
:1009E00079202020202020203A200046292046611E
:1009F000696C736166652064656C617920202020D4
:100A00002020203A200050574D206368616E6E65AB
:100A10006C200066756E6374696F6E3A2000292041
:100A2000706F72742000506F776572546F776572C3
:100A300000445446205548462033322D62697420C4
:100A400031306368004F70656E4C52536E67525878
:100A5000206D696E6920342F36636800466C7974A6
:100A6000726F6E2F4F72616E6765525820554846FF
:100A70002038636800525820747970653A20004429
:100A8000697361626C656400487A00203D3D200016
:100A900043616C63756C61746564207061636B6540
:100AA0007420696E74657276616C3A200042292068
:100AB0004D6963726F202868616C66292050504D23
:100AC000202020203A00412920496E766572746505
:100AD000642050504D20696E20202020203A0030A4
:100AE00029204D7574652062757A7A657220286DAB
:100AF0006F73746C79293A003929205365726961E2
:100B00006C2062617564726174653A00736D617224
:100B100074506F7274004672536B79005472616E38
:100B200073706172656E740044697361626C6564B0
:100B30000038292054656C656D657472793A2020FF
:100B40002020202020003729204368616E6E656CCC
:100B500020636F6E6669673A202000362920446161
:100B60007461726174652028302D32293A2020206A
:100B700000352920486F70206368616E6E656C7364
:100B80003A2020202020003429204368616E6E65C1
:100B90006C2073706163696E673A202000332920EE
:100BA000524620706F7765722028302D37293A2001
:100BB0002020003229205246206D616769633A2067
:100BC0002020202020202020003129204261736530
:100BD000206672657175656E63793A202020000089
:100BE00000000700020100000304060000000000EE
:100BF00000000001020408102040800102040810D7
:100C00002001020408102004040404040404040263
:100C10000202020202030303030303000000002395
:100C2000002600290000000000250028002B0000FD
:100C3000000000240027002A0000872D11241FBE79
:100C4000CFEFD8E0DEBFCDBF13E0A0E0B1E0ECE134
:100C5000F1E602C005900D92A83CB107D9F716E065
:100C6000A8ECB3E001C01D92AE38B107E1F71CE07B
:100C7000CCE3DCE004C02297FE010E94902ECA3330
:100C8000D107C9F70E94C32D0C948C300C9400003E
:100C900080917305813019F482E08093730580910F
:100CA0007305833019F484E0809373050895A89543
:100CB0000895DC01ED91FC910190F081E02D099502
:100CC00008952091740530917505382748E0C901D1
:100CD000880F991F37FF06C09C0151E2252750E17C
:100CE000352701C09C01415091F730937505209341
:100CF0007405089588E38093760580E092ECA1E086
:100D0000B0E08093770590937805A0937905B09330
:100D10007A0587E08093830580EC92E9ADEEB9E136
:100D200080937B0590937C05A0937D05B0937E0511
:100D300085E0809384058DEE9EEFADEABEED809355
:100D40007F0590938005A0938105B0938205E5E827
:100D5000F5E080E090E0863028F4DC01AE54BC4F32
:100D60002C9101C020E0219301968831910599F7DB
:100D700082E080939D058AE080939E05089580EC33
:100D800091EDA8E9BBE18093BB059093BC05A093CE
:100D9000BD05B093BE0580E090E0A0E0B0E5809393
:100DA000BF059093C005A093C105B093C205E3ECC5
:100DB000F5E080E081938F5F8031E1F70895A0E056
:100DC000B0E0E5EEF6E00C94592ED82F0E94BE2834
:100DD0006115710581059105C9F30E94FC2E1092E1
:100DE0007F05109280051092810510928205C4E063
:100DF000812C912C54018A94C0907F05D09080055D
:100E0000E0908105F0908205FE2CED2CDC2CCC24AA
:100E10000E94F72EA50194010E94382E6C0D7D1DB5
:100E20008E1D9F1D60937F057093800580938105C3
:100E300090938205C15001F7DD2309F450C005E805
:100E400015E0E801A12CB12C62E3C62ED12CE12CD7
:100E5000F12C8881882309F442C0B39419F40E94CC
:100E60007A063DC00E94F72EA70196010E94382EF7
:100E7000E1E0E60FA5E8B5E08A2F801B8A1520F493
:100E80008D918E13F9CFE9CF2091840530E0A0E158
:100E9000B7E20E94D02D9B01AC01AE2FB0E00E94C2
:100EA000DF2D40907B0550907C0560907D05709013
:100EB0007E05640D751D861D971D4090BB055090E5
:100EC000BC056090BD057090BE05461657066806C5
:100ED000790618F2E993A39488E1A812BACFCDB7A6
:100EE000DEB7E0E10C94752E8436910520F4BC0148
:100EF00080E090E017C09C018E3B910528F42A55B4
:100F00003109AAE0B0E00CC0823D910528F4245BD1
:100F10003109A4E6B0E004C02D5C3109A8E5B2E0D7
:100F20000E94D02DA4E6B0E09B01AC010E94DF2D11
:100F3000089590E08C599F4F0E947407089561E0D6
:100F400083E10E946B2960E083E10E94A42982E092
:100F50008093B00085E08093B10061E083E00E945F
:100F60006B2960E083E00E94A4290895A4E0B0E02A
:100F7000ECEBF7E00C94672E009749F19C0140E000
:100F800050E068E478EE81E090E00E94382E61E065
:100F900083E129833A834B835C830E94A4292981BE
:100FA000822F3A81932F4B81A42F5C81B52F8F3FE5
:100FB0009105A105B10529F020F08FEF90E0A0E0A8
:100FC000B0E08093B3008091B000806107C060E022
:100FD00083E10E94A4298091B0008F7E8093B000AD
:100FE0002496E2E00C94832E60E08CE00E946B2952
:100FF00061E08BE00E946B2961E08DE00E946B292B
:1010000060E082E00E946B2961E084E00E946B292D
:10101000089542E050E068E476E080E00E94EE2728
:101020000895E3E0F0E089E080935700E491E670F2
:1010300081E0E63009F080E00895CF93DF93C82F78
:101040000E941108882381F0DFB781E08093720548
:10105000F8940E94570688E180936000C093600076
:10106000C1110E945706DFBFDF91CF9108958F9283
:101070009F92AF92BF92CF92DF92EF92FF92CF9367
:10108000FC01C0A5EC2FE770F0E0E658FC4FA08112
:10109000B0E0C7FF03C024E130E002C02FE030E041
:1010A000FC0197A183E1989FF0011124E25CFE4FBF
:1010B00080809180A280B380A20FB31F20E43FE123
:1010C0004DE750E00E94EA2DA50194010E94162EE2
:1010D0008C2F887149F469017A01E0EDCE0EE7E0CA
:1010E000DE1EE11CF11C1BC0C7FF05C060E47AE8EE
:1010F0008CE29EE004C060E07EEE8AEB9BE069013A
:101100007A01F8EBCF0EFBE0DF1EE11CF11CA5011C
:1011100094010E94162EC20ED31EE41EF51EC701B6
:10112000B60169517C4F8F4F9F4F28EE33E040E06E
:1011300050E00E94162EA8EEB3E00E94DF2DCF9162
:10114000FF90EF90DF90CF90BF90AF909F908F90E7
:1011500008958F3F910551F048F0811522E09207E4
:1011600038F08115934030F482E0089580E00895CE
:1011700081E0089583E00895A0E0B0E0E2ECF8E0BB
:101180000C94622EEB018A01B82FB695A0E028815D
:101190003981F80120832A813B8121832C813D8183
:1011A00022832E813F812383688179814A815B81FB
:1011B0002C813D81EE81FF819F2F9295990F990F90
:1011C000907C272F2370922B252F2370220F220F24
:1011D000922B232F23702295207F922BF80194834A
:1011E0000B5F1F4F2896AF5FBA1788F680FF24C0A9
:1011F000888199810E94A908D82E8A819B810E94AA
:10120000A908E82E8C819D810E94A908F82E8E8164
:101210009F810E94A908F0E4DF9EA001112490E1C3
:10122000E99E90011124242B282BE4E0FE9EB001BE
:101230001124262BF8012083CDB7DEB7E7E00C940C
:101240007E2E803223E0920708F1883E23E0920749
:1012500040F48F519340E4E096958795EA95E1F745
:101260000895803D27E0920718F48C5D934008951F
:10127000883928E0920768F4885C974074E0969576
:1012800087957A95E1F78D509C4F089580E090E026
:1012900008958FEF93E008958C30910540F4A4E019
:1012A000880F991FAA95E1F7885D9C4F0895843FA8
:1012B00023E0920718F484529C4F0895811524E08E
:1012C000920740F48657934FF4E0880F991FFA95E0
:1012D000E1F7089580E998E008959C0136952795F7
:1012E00025753575821B930B9C012373337396957B
:1012F00087959695879583739373820F931F9C01AF
:1013000054E0369527955A95E1F7280F391F2F702D
:101310003F7041E051E0249FC001259F900D349F14
:10132000900D1124892F08952D98882319F000001D
:101330002B9A02C000002B9800002D9A00000895FF
:101340002D9A000083B12D98000082958170089538
:10135000CF93DF93D82F5C9A2D985C98C8E08D2F9F
:1013600080780E949409DD0FC150C9F72D98DF9154
:10137000CF9108958F770E94A8090895CF93DF93A6
:10138000D82FC8E08D2F80780E949409DD0FC150BE
:10139000C9F72D98DF91CF910895CF93DF932D98C2
:1013A000C8E080E0D82FDD0F0E94A0098D0FC1504A
:1013B000C9F7DF91CF9108950E94BA090E94CD0923
:1013C0005C9A0895A1E0B0E0E8EEF9E00C94672E95
:1013D000806869830E94A8096981862F0E94BE09DE
:1013E0005C9A2196E2E00C94832ECF93C0917F0506
:1013F000C827E82FF0E0EA58FA4F678589E70E948E
:10140000E2096C2F8DE30E94E2096C2F82E40E94B6
:10141000E209CF91089586E20E94DC090895CF93F6
:10142000DF93EC016C818CE10E94E2096D818DE11A
:101430000E94E2096E818EE10E94E2096F8180E2E2
:101440000E94E209688581E20E94E209698582E2E0
:101450000E94E2096A8583E20E94E2096B8584E2C8
:101460000E94E2096C8585E20E94E2096D858AE2AC
:101470000E94E2096E858EE60E94E2096F858FE682
:101480000E94E209688980E70E94E209698981E790
:101490000E94E2096A8982E70E94E209DF91CF9106
:1014A0000895CF92DF92EF92FF92CF93DF936B017B
:1014B0007C01C11488E3D8068CE9E8068CE1F806C3
:1014C00028F5C701B60120E836E948E950E00E9456
:1014D000162EE901689760E879E687E69FEF0E949B
:1014E000F22D6C0D7D1D8E1D9F1DF2E0660F771F86
:1014F000881F991FFA95D1F721E732E040E050E0CC
:101500000E94162EF22EE32E80E421C0C701B60100
:1015100020E03DE241E351E00E94162EE901689788
:1015200060E073ED8EEC9EEF0E94F22D6C0D7D1D40
:101530008E1D9F1D660F771F881F991F21E732E0C0
:1015400040E050E00E94162EF22EE32E80E66C2F33
:101550006F71680F85E70E94E2096E2D86E70E9491
:10156000E2096F2D87E70E94E209DF91CF91FF909A
:10157000EF90DF90CF900895682F8DE60E94E209EA
:1015800008958F929F92AF92BF92CF92DF92EF9287
:10159000FF92CF93DF93D82F83E00E94DC098093E2
:1015A000710584E00E94DC098093700560E086E0AC
:1015B0000E94E20961E087E00E94E2096FE789E0AA
:1015C0000E94E20965E08AE00E94E20962E18BE0A4
:1015D0000E94E20965E18CE00E94E2096DEF8DE076
:1015E0000E94E20960E08EE00E94E209DD2319F02A
:1015F0008BE291E008C020919D0533E1239FC0015B
:101600001124825C9E4F0E940F0A6CE880E30E94C6
:10161000E2096FE082E30E94E20962E483E30E9450
:10162000E20980919E0587FF02C064E101C06AE083
:1016300084E30E94E2096AE285E30E94E2096DE226
:1016400086E30E94E20964ED87E30E94E20960E01C
:1016500088E30E94E20960E089E30E94E209D11177
:1016600009C0C0907F05D0908005E0908105F09082
:10167000820507C0C5E9CC2EC1ECDC2EED2CCEEDE9
:10168000FC2ECAE38F2C9924AA24BB24682D8C2F0E
:101690000E94E209682D85E08C0F0E94E209FE2C71
:1016A000ED2CDC2CCC24CF5FCE3361F76FEF83E4DD
:1016B0000E94E2096FEF84E40E94E2096FEF85E483
:1016C0000E94E2096FEF86E40E94E209DD2311F037
:1016D00066E002C0609183058DE60E94E20960E049
:1016E00089E70E94E209609184058AE70E94E20985
:1016F00060E083E70E94E20960E084E70E94E2097B
:10170000D11109C060917B0570917C0580917D05A8
:1017100090917E0504C060EC72E98DEE99E10E9423
:10172000510ADF91CF91FF90EF90DF90CF90BF9063
:10173000AF909F908F90089561E087E00E94E2094A
:1017400064E28EE70E94E20963E088E00E94E20919
:1017500060E088E00E94E20965E087E00E94E2091B
:1017600062E085E00E94E20983E00E94DC09809348
:10177000710584E00E94DC0980937005089583E080
:101780000E94DC098093710584E00E94DC0980934B
:10179000700561E087E00E94E2096AE070E080E0A5
:1017A00090E00E94E1280E949C0B00000895CF92D7
:1017B000DF92FF920F931F93CF93DF931F92CDB7CA
:1017C000DEB7082F162F8EE399830E94E209F02ED0
:1017D000C02E9981D92E8C2D8F19811738F4F601DE
:1017E00061916F018FE70E94E209F5CF64E085E027
:1017F0000E94E20983E00E94DC098093710584E085
:101800000E94DC09809370050E94BE2860936C05DD
:1018100070936D0580936E0590936F0569E087E086
:101820000E94E20981E0809373050F90DF91CF91D0
:101830001F910F91FF90DF90CF9008950F931F930A
:101840000E94D70B80917305813099F40E94BE28C5
:1018500000916C0510916D0520916E0530916F051A
:10186000601B710B820B930B603A764881409105A7
:1018700048F380917305813031F46EE971E082EEB6
:1018800095E00E94AA2A1F910F9108950F931F932C
:1018900080917305823021F41092730581E020C09D
:1018A000809173058130D9F40E94BE2800916C05A7
:1018B00010916D0520916E0530916F05601B710BC5
:1018C000820B930B613A76488140910540F061E0CC
:1018D00087E00E94E2091092730582E001C080E077
:1018E0001F910F910895CF93DF93EC014AE050E0F0
:1018F0006D2F70E082EE95E00E94782B6EE282EE12
:1019000095E00E947C2ABE0184E0769567958A95D1
:10191000E1F76F7077274AE050E082EE95E00E9491
:10192000782BDF91CF910895D82FC0E0CD1790F498
:101930005E9A409A64E670E080E090E00E94E128C0
:101940005E98409864E670E080E090E00E94E128B4
:10195000CF5FECCF6CE271E080E090E00E94E12884
:10196000E4CF0F931F93CF93DF93EC01062F15E085
:10197000115051F0CE010E947330081741F0602FD2
:10198000CE010E947B30F4CF82E00E94940CDF9164
:10199000CF911F910F910895A0E0B0E0E2EDFCE03F
:1019A0000C94592E482E562EC0E0D0E0612C712C9C
:1019B000E12CF12C00E010E041100CC06090D40547
:1019C00086E4689E3001112459E1E52EF12C0AEBE2
:1019D00015E01EC091E049120FC06090D405E6E406
:1019E0006E9E30011124FBE16F0E711C49E2E42E62
:1019F000F12C06E715E00CC082E0481209C028E18E
:101A0000622E77247394EE24E394F12C03ED15E019
:101A100043018C0E9D1E10927505109274053401C1
:101A2000A62CA818B12CC30101966C01AE14BF04FA
:101A3000A8F4A00EB11E511006C0C3010E9473305D
:101A4000F501808305C0F5016081C3010E94B10CDE
:101A5000F50180810E9461063601E2CFC301511079
:101A600018C0C3010E947330B82EC6010E947330A3
:101A70002B2D30E0322F2227282B80917405909156
:101A800075058217930779F4C0E0D0E0552453948C
:101A900093CF3601609175050E94B10C6091740579
:101AA000C6010E94B10CC05EDE4FC13E92E0D90774
:101AB00008F482CF852DCDB7DEB7E0E10C94752E0A
:101AC00061E082E00E94CC0C089560E082E00E9418
:101AD000CC0C8091D305853028F084E08093D30529
:101AE0000E94600D8091D3058093D405089561E034
:101AF00080E00E94CC0C61E081E00E94CC0C089553
:101B000060E080E00E94CC0C882351F060E081E02E
:101B10000E94CC0C882321F080917605883349F00F
:101B20000E94BF060E947A0681E00E94DF060E94A2
:101B3000770D0895882319F06AEA71E002C06EEA11
:101B400071E082EE95E00E94AA2A0895FF920F9319
:101B50001F93CF93DF9369EC7BE082EE95E00E94C8
:101B6000562A40917B0550917C0560917D057091CE
:101B70007E052AE030E082EE95E00E947F2B63EB49
:101B80007BE082EE95E00E94562A40917F055091BD
:101B90008005609181057091820520E130E082EE40
:101BA00095E00E947F2B6DE97BE082EE95E00E943C
:101BB000562A4AE050E06091830582EE95E00E944B
:101BC000A72B67E87BE082EE95E00E94562A4AE068
:101BD00050E06091840582EE95E00E94A72B61E7BA
:101BE0007BE082EE95E00E94562AC5E8D5E0F12C14
:101BF0008E0188818823A9F0FF2031F061EB71E02C
:101C000082EE95E00E94792A21964AE050E0F801A0
:101C1000608182EE95E00E94702BF394F8E1FF1250
:101C2000E7CF82EE95E00E94842A6BE57BE082EEAE
:101C300095E00E94562A4AE050E060919D0582EEB0
:101C400095E00E94A72B66E47BE082EE95E00E947F
:101C5000562AE0919E05E770F0E0EE0FFF1FEE5769
:101C6000FC4F6081718182EE95E00E94AA2A61E3B7
:101C70007BE082EE95E00E94562A80919E05887155
:101C8000883069F028F4811113C068E27BE00CC051
:101C9000803141F0883161F46CE07BE005C06CE19B
:101CA0007BE002C066E17BE082EE95E00E94982A2C
:101CB00068EF7AE082EE95E00E94562A409177051F
:101CC000509178056091790570917A052AE030E0AD
:101CD00082EE95E00E947F2B6FED7AE082EE95E038
:101CE0000E94562A8091BF0580710E949A0D66EC71
:101CF0007AE082EE95E00E94562A8091BF058074BA
:101D00000E949A0D6DEA7AE082EE95E00E94562AD2
:101D10008091BF0580720E949A0D60E97AE082EEA0
:101D200095E00E94562A86E795E00E943708AB01AD
:101D3000BC012AE030E082EE95E00E94612B6BE866
:101D40007AE082EE95E00E94562A86E795E00E94AE
:101D500037089B01AC0160E472E48FE090E00E94E0
:101D6000162EBA01A9012AE030E082EE95E00E9429
:101D7000612B68E87AE082EE95E00E94982ACDB760
:101D8000DEB7E5E00C94802E8F929F92AF92BF92C7
:101D9000CF92DF92EF92FF92811107C06FE77AE056
:101DA00082EE95E00E94982A2FC090E00E9474076E
:101DB00024E630E040E050E00E94162ECA01B9014E
:101DC0002AE030E040E050E00E94162E49015A011E
:101DD0006B017C012AE030E0B501A40182EE95E0C0
:101DE0000E94612B6EE282EE95E00E947C2A2AE03E
:101DF00030E0B701A60182EE95E00E94612B63E717
:101E000082EE95E00E94BC2AFF90EF90DF90CF9089
:101E1000BF90AF909F908F9008951F93CF93DF93C3
:101E200065E77AE082EE95E00E94562A80919F0550
:101E3000813041F46CE57AE082EE95E00E94982AC8
:101E400010E050C0823019F465E47AE0F5CF8430B8
:101E500019F461E37AE0F0CF853091F766E27AE039
:101E6000EBCFC12FD0E0C930D1050CF441C068E3FD
:101E7000610F82EE95E00E947C2A6EE17AE082EEAC
:101E800095E00E94562ABE016F5F7F4F4AE050E006
:101E900082EE95E00E94402B63E17AE082EE95E0CD
:101EA0000E94562AC156DA4FE981E03218F566E001
:101EB0007AE082EE95E00E94562A8981803130F0E6
:101EC0006DE673E082EE95E00E94792A69816F7079
:101ED00070E06F5F7F4F4AE050E082EE95E00E9435
:101EE000492B1F5F80914805181708F4BACF0FC01F
:101EF00061E3BECFEF70F0E0EE0FFF1FEE56FC4F38
:101F00006081718182EE95E00E94AA2AEACF6BEE91
:101F100079E082EE95E00E94562A8091B7050E94F2
:101F2000C40E60ED79E082EE95E00E94562A809121
:101F3000B8050E94C40E65EB79E082EE95E00E9440
:101F4000562A8091B9050E94C40E6AE979E082EEB2
:101F500095E00E94562A4091AF055091B0056091DE
:101F6000B1057091B205411551056105710539F151
:101F70002AE030E082EE95E00E947F2B67E679E070
:101F800082EE95E00E94562A8091B3050E9499073F
:101F9000AB01BC012AE030E082EE95E00E947F2B8D
:101FA00063E479E082EE95E00E94562A4AE050E030
:101FB0006091B40582EE95E00E94A72B06C06AE30B
:101FC00079E082EE95E00E94982A6DE179E082EE58
:101FD00095E00E94562A6091B5057091B6054AE0D9
:101FE00050E082EE95E00E94912B60E079E082EE75
:101FF00095E00E94562A6091AE05603450F470E07E
:102000006F5F7F4F4AE050E082EE95E00E94492BDF
:1020100006C067EF78E082EE95E00E94982A6AEDAC
:1020200078E082EE95E00E94562A8091AD0580FF0F
:1020300003C063EB71E002C067EB71E082EE95E0F4
:102040000E94AA2A6DEB78E082EE95E00E94562A63
:102050008091AD0582700E949A0D6EE978E082EE63
:1020600095E00E94562A8091AD0584700E949A0DD9
:102070006FE778E082EE95E00E94562A8091AD05E8
:1020800088700E949A0DDF91CF911F9108950F9350
:102090001F93CF93DF93209145052F3FA9F56FEF55
:1020A00075E082EE95E00E94562A80E893E00E9457
:1020B000730C6EED75E082EE95E00E94562A8091D9
:1020C0004605909147050E94730C6BEA75E082EE1D
:1020D00095E00E94982A68E875E082EE95E00E94FB
:1020E000982A60E775E082EE95E00E94982A6BE4FA
:1020F00075E082EE95E00E94982A82EE95E00E94BB
:10210000842A0E940D0F68C012160CF065C0332798
:1021100027FD30958091480590E0821793070CF4D5
:102120005BC066E375E082EE95E00E94562A6091FE
:102130004505772767FD70954AE050E082EE95E00F
:102140000E94492B6BE075E082EE95E00E94562AD2
:1021500010E008E2809149051817D0F5C12FD0E0B2
:10216000CC0FDD1FC65BDA4F288130E0809145053A
:10217000992787FD909501972817390739F56BEB5B
:1021800071E082EE95E00E94792A4AE050E0602FEB
:1021900082EE95E00E94702B6FEB71E082EE95E08D
:1021A0000E94792AE981EF70F0E0EE0FFF1FEE56F2
:1021B000FC4F6081718182EE95E00E94792A63EC88
:1021C00071E082EE95E00E94792A0F5F1F5FC2CF17
:1021D00082EE95E00E94842ADF91CF911F910F91AA
:1021E0000895FF920F931F93CF93DF93C5E8D5E037
:1021F000F12C8E0188818823D1F165EC71E082EEAB
:1022000095E00E94792A4AE050E06F2D82EE95E039
:102210000E94702B62ED71E082EE95E00E94792AB7
:102220002196F801208130E0A0E1B7E20E94D02D94
:102230009B01AC01A0918405B0E00E94DF2DAB01B1
:10224000BC0180917B0590917C05A0917D05B091AA
:102250007E05480F591F6A1F7B1F2AE030E082EE7F
:1022600095E00E947F2BF394F8E1FF12C2CFCDB727
:10227000DEB7E5E00C94802E1092DF0485E6E0EEF8
:10228000F4E0DF011D928A95E9F70895CF93C82FF6
:102290008F3719F0883009F045C0E091DF04EE2354
:1022A000D9F1E150E093DF04F0E0E052FB4F1082FF
:1022B0006DE070E082EE95E00E945906C0E08091EA
:1022C000DF04C81760F4EC2FF0E0E052FB4F6081B0
:1022D00070E082EE95E00E945906CF5FF0CF60E299
:1022E00070E082EE95E00E9459066DE070E082EEAB
:1022F00095E00E945906C0E08091DF04C81778F588
:10230000EC2FF0E0E052FB4F608170E082EE95E050
:102310000E945906CF5FF0CF67E082EE95E00E9401
:102320007C2A1DC08B3119F40E943C111AC08D30DB
:10233000C1F08A30B1F08091DF04843668F76C2FE9
:1023400070E082EE95E00E945906E091DF0481E0A2
:102350008E0F8093DF04F0E0E052FB4FC08380E0FB
:1023600001C081E0CF910895CF93C82F0E94BE286D
:102370006093C8047093C9048093CA049093CB04FB
:10238000C093DD04CC2329F040E051EE60E070E022
:1023900004C040E855E260E070E082EE95E00E9403
:1023A000062DCF9108959091CC04492F4F7050E0A5
:1023B000BA016F5F7F4F292F30E0E4E03595279514
:1023C000EA95E1F76217730759F0FA01E353FB4FFF
:1023D000808381E0890F8F70907F892B8093CC045C
:1023E00008956EE770E082EE95E00E945906089528
:1023F000A3E1B1E0EEEFF1E10C945A2EE5E8F5E04F
:10240000712C8191882321F0739428E17212F9CF05
:1024100066ED71E082EE95E00E94AA2A4AE050E063
:10242000672D82EE95E00E94A72B80E00E94C10AF2
:102430000E949C0B8E010E5F1F4FC12CD12C760188
:10244000C39466246A945C2C0E94B2284B015C0100
:102450002091840530E0A0E1B7E20E94D02D9B01DD
:10246000AC01C701B6010E94F22D20917B0530918D
:102470007C0540917D0550917E05620F731F841F7E
:10248000951F2091BB053091BC054091BD05509131
:10249000BE05261737074807590718F4F801608268
:1024A00029C08C2D0E94F50961E070E080E090E089
:1024B0000E94E128F80110820E94B2286819790967
:1024C0008A099B09643F71408105910540F40E948F
:1024D0000B0AF8019081981778F78083EDCF50FEB2
:1024E00005C05D9841985E9A409A04C05D9A419AF1
:1024F0005E9840982FEFC21AD20AE20AF20A0F5FE2
:102500001F4F8FEFC816D104E104F10409F09BCFEF
:10251000CE019395FC01D82E7FEF68EC2E2F281B5F
:10252000271510F051E056C0DE01129651E02FEF52
:1025300041E03D91321710F0322F01C0452F5F5F0F
:102540005F3F11F0232FF5CF4193242F30E0A1E01E
:10255000B0E0AC0FBD1FA20FB31F5C93413079F008
:10256000DE01A20FB31F5C93423049F0AFEFBFEF23
:10257000AC0FBD1FA20FB31F6C934E3F78F6A2E0C5
:10258000B0E0AC0FBD1FA20FB31F7C934D3F30F6E0
:10259000A3E0B0E0AC0FBD1FA20FB31F6C93BECF82
:1025A000452F242F30E0FC01E20FF31F6081AFEFD5
:1025B000B0E0AC0FBD1FA20FB31F2C91621748F4FF
:1025C0004150DC01A40FB11D2C9120836C9341116B
:1025D000E8CF5F5F571520F3372D369520E023179E
:1025E00070F4DC01A20FB11D4C91522F530FFC016E
:1025F000E50FF11D50815C9340832E5FF0CFF5E82D
:10260000EF2EF5E0FF2E8C01802F8D19871598F4A1
:10261000F801C1908F014AE050E06C2D82EE95E008
:102620000E94702B6CE282EE95E00E947C2AF701FA
:10263000C1927F01E9CF82EE95E00E94842A81E079
:10264000CD5EDE4FEFE00C94762E1F920F920FB608
:102650000F9211241F932F933F934F935F936F9388
:102660007F938F939F93AF93BF93CF93DF93EF931A
:10267000FF93C0918600D09187008091870490914C
:1026800088042091A904211155C09E01281B390BF3
:102690008091BF059091C005A091C105B091C20580
:1026A00085FD02C036952795253C49E03407B8F1F1
:1026B00040910A0150E060E070E02CE1B695A795EA
:1026C000979587952A95D1F70097A105B10521F433
:1026D00081E090E0A0E0B0E084179507A607B70777
:1026E000D8F480910A018F3FB9F040E080910A014F
:1026F000481780F4842F90E0880F991FFC01E7575A
:10270000FB4F20813181FC01E55FFE4F3183208347
:102710004F5FECCF1092AA0410920A010BC02D3B20
:1027200082E0380720F080910A018031D8F08FEFE5
:1027300080930A01D0938804C0938704FF91EF919E
:10274000DF91CF91BF91AF919F918F917F916F91C9
:102750005F914F913F912F911F910F900FBE0F905E
:102760001F90189510910A0181E0810F80930A0152
:10277000C9010E942109E12FF0E0EE0FFF1FE7578A
:10278000FB4F91838083D6CF83E0809380008AE9DA
:10279000809381008091BF0586FD05C080918100F6
:1027A0008064809381008FEF9FEF909389008093E6
:1027B000880080916F00806280936F0008950E946E
:1027C000650D8091D405843011F41092D4050895DC
:1027D0006F3018F086958058089589E0689F802DA5
:1027E00011240895A0E0B0E0E8EFF3E10C94612E2D
:1027F000C82F0E94BE2800913804109139042091FE
:102800003A0430913B046B017C01C01AD10AE20A00
:10281000F30A9701860149E8C41643E1D406E104AE
:10282000F10410F010923C04609338047093390462
:1028300080933A0490933B042091A9048FEF820F78
:102840008230D8F5E0913C04EE2309F44EC1E1302A
:1028500011F482E0B8C1E03108F034C181E08E0F9C
:1028600080933C04F0E0E757FB4FC083803109F0D0
:10287000ACC1EBE8F4E0213029F4A181A695A6953E
:10288000808108C080819181A92FA695A695A695E3
:1028900096958795A03148F4B0E090E0AA0FBB1F51
:1028A000A55FBE4F11969C938E931092AA04329608
:1028B00084E0E939F807F9F688C1233009F005C149
:1028C000E0913C04E11104C0CF3009F07EC10DC19C
:1028D000E83148F481E08E0F80933C04F0E0E85743
:1028E000FB4FC08372C1E83109F0ECC0C111EAC0EE
:1028F00040E050E0ABE0CA01B3E0880F991FBA9501
:10290000E1F7A49F9001A59F300D1124F901E7572D
:10291000FB4F6081E1817E2F777075956795FC0193
:10292000EE0FFF1FE55FFE4F71836083F901E657ED
:10293000FB4FB081B695B695B695E181FE2FF29525
:10294000FF0FF07E6F2F6B2BE695E695E6957E2FB9
:10295000777075956795FC01EE0FFF1FE35FFE4FE3
:1029600071836083F901E557FB4FB081B295B6954D
:10297000B695B370C181DC2FDD0FDD0F6D2F6B2B92
:10298000C295C695C695C370E281E170EE0FEE0F59
:102990007E2F7C2B75956795FC01EE0FFF1FE15F85
:1029A000FE4F71836083F901E357FB4FB081B69509
:1029B000E181FE2FF795FF27F7956F2F6B2BE6959B
:1029C0007E2F777075956795FC01EE0FFF1FEF5E08
:1029D000FE4F71836083F901E257FB4FB081B295DE
:1029E000BF70E181FE2FF295F07F6F2F6B2BE29588
:1029F000EF707E2F777075956795FC01EE0FFF1FC6
:102A0000ED5EFE4F71836083F901E157FB4FB081AA
:102A1000BB1FBB27BB1FC181DC2FDD0F6D2F6B2BB5
:102A2000CC1FCC27CC1FE281E370EE0F7E2F7C2BD6
:102A300075956795FC01EE0FFF1FEB5EFE4F7183EE
:102A40006083F901EF56FB4FB081B695B695E181F1
:102A5000FE2FF295FF0FFF0FF07C6F2F6B2BE6958B
:102A6000E6957E2F777075956795FC01EE0FFF1F39
:102A7000E95EFE4F71836083F901EE56FB4F2081C2
:102A80002295269527703181E32FEE0FEE0FEE0F82
:102A90006E2F622B732F729576957770759567956B
:102AA000FC01EE0FFF1FE75EFE4F718360834F5FF7
:102AB0005F4F4230510509F01ECF80919F0483FF84
:102AC0001092AA0410923C0480C0243009F07DC00A
:102AD00060913C0461110BC0C83AB1F410927505C5
:102AE0001092740588EA0E94610681E06CC0613032
:102AF00019F4C093370404C0623031F4C093360433
:102B00008C2F0E9461065AC0E09136042E2F30E0CF
:102B1000220F331F462F50E0C901029684179507F4
:102B20003CF0633268F7FA01EA57FB4FC083E8CF05
:102B30002D5F3F4F8C2F90E060917405709175056B
:102B40004217530749F4982F882786279727909391
:102B500075058093740532C06817790769F580910F
:102B60003704813049F5E13118F080E18093360473
:102B7000F0903604CAE8D4E000E010E00F15D0F47D
:102B8000FE013197808190E0982F88272881822B41
:102B900063E0969587956A95E1F70E942109F8010F
:102BA000EE0FFF1FE55FFE4F918380830F5F1F4F86
:102BB0002296E4CF1092AA0410923C0480913C0427
:102BC000882319F08F5F80933C04CDB7DEB7E8E02F
:102BD0000C947D2EE82FF0E0E654FA4FE185E031C9
:102BE00050F4F894F0E0EE0FFF1FE55FFE4F808198
:102BF000918178940895E03121F0E13131F483E15D
:102C000001C082E10E94002A089580E092E00895C8
:102C1000A2E2B0E0EEE0F6E10C94572E9E012F5FA9
:102C20003F4F80E1D9011D928A95E9F764E072E097
:102C300082EE95E029A33AA30E94AA2A0E94BF0B24
:102C40001D8A1E8A1F8A188E312C212C00E0812CAF
:102C5000912C540170E4472E71EE572E7DE9672EBA
:102C600078E1772EE0E5CE2EE3ECDE2EE12CF12CA0
:102C700084EF91E0A0E0B0E08D8F9E8FAF8FB8A37E
:102C800080EC91EDA8E9BBE1898F9A8FAB8FBC8F67
:102C900080E491EEADE9B8E1898B9A8BAB8BBC8B6C
:102CA00082EE95E00E94BE2B892B09F4E1C082EEF2
:102CB00095E00E94EB2B9C0133272C32310509F45F
:102CC00042C0ACF42332310509F0ABC019821A823C
:102CD0001B821C821D821E821F82188619861A86FC
:102CE0001B861C861D861E861F86188A60C024349B
:102CF000310529F02335310509F4B2C092C064E4EE
:102D000082EE95E00E947C2A2AE030E040E451EE19
:102D10006DE978E182EE95E00E940A2B6CE282EE8A
:102D200095E00E947C2A2AE030E040EC51ED68E911
:102D30007BE182EE95E00E940A2B6CE282EE95E048
:102D40000E94BC2AADCF0F5F043009F0A9CF2981C2
:102D50003A814B815C81A8EEB3E00E94DF2D698B44
:102D60007A8B8B8B9C8B2D813E814F8158850E9465
:102D7000DF2D698F7A8F8B8F9C8F29853A854B85C4
:102D80005C852D8F3E8F4F8F58A32D853E854F85B7
:102D900058890E94DF2D6B017C0160323EE473078D
:102DA0008105910530F462E38CE10E94E20900E0C4
:102DB00077CF603345E774078105910510F462E22F
:102DC000F3CF60345CE975078105910510F466E284
:102DD000EBCF80E5C81683ECD806E104F10410F4CB
:102DE00062E1E2CF90E6C9169AEED906E104F10459
:102DF00010F465E1D9CFA0E7CA16A1E1DA06A1E097
:102E0000EA06F10410F461E0CFCFB0EACB16B6E8E1
:102E1000DB06B1E0EB06F10410F463E0C5CF65E03A
:102E2000C3CF10ED180F1A3008F03ACFE1E0F0E010
:102E3000EC0FFD1F24E0029FE00DF11D1124208105
:102E4000318142815381AAE0B0E00E94DF2D610F01
:102E5000711D811D911D608371838283938320CFB7
:102E600049885A886B887C88812C912C540118CF12
:102E700081149104A104B10489F4C301B2010E9438
:102E8000510A61E070E080E090E00E94E1281D8A34
:102E90001E8A1F8A188E312C22242A948D8D9E8D95
:102EA000AF8DB8A188169906AA06BB06D0F40E9479
:102EB0000B0A2D893E894F89588D280F311D411DE0
:102EC000511D2D8B3E8B4F8B588F381608F4382EA2
:102ED000821508F4282E3FEF831A930AA30AB30A37
:102EE00056C0C301B20128EE33E040E050E00E943A
:102EF000162EBA01A9012AE030E082EE95E00E9488
:102F0000612B6CE282EE95E00E947C2A4AE050E060
:102F1000632D82EE95E00E94702B6CE282EE95E0CC
:102F20000E947C2A6D897E898F89988DA5019401E4
:102F30000E94162EBA01A9012AE030E082EE95E047
:102F40000E94612B6CE282EE95E00E947C2A4AE0AE
:102F500050E0622D82EE95E00E94702B6CE282EED2
:102F600095E00E94BC2A4C0C5D1C6E1C7F1C898D58
:102F70009A8DAB8DBC8D84159505A605B70520F4FB
:102F800049885A886B887C88812C912C5401298926
:102F90003A894B895C89283E33404105510509F047
:102FA0007FCEA296E2E10C94732EACE1B0E0EBEDA3
:102FB000F7E10C94612E0E94BE286B017C0181E038
:102FC0000E94C10A14E703E0198361E0CE01019673
:102FD0000E941E0C009373050E949C0B6AEF70E028
:102FE00080E090E00E94E12880917305833089F4AD
:102FF00082EE95E00E94BE2B892B59F40E94BE28D8
:103000006C197D098E099F096038734C894C914079
:10301000D8F280917305833009F44FC08FE70E9486
:10302000BA090E94CD098983843511F083E05CC020
:103030000E94CD0910924605809347050E94CD0954
:103040002091460530914705280F311D30934705E3
:10305000209346050E94CD09809348050E94CD0922
:1030600080934905813110F7F12C0F2D10E08091EC
:10307000490590E0880F991F0817190740F40E942E
:10308000CD09F801E65BFA4F8083F394EECF80E739
:10309000898361E0CE0101960E941E0C83E080933B
:1030A00073050E949C0B62E370E080E090E00E9458
:1030B000E12880917305833011F482E015C08FE719
:1030C0000E94BA090E94CD098983803509F0AECFEC
:1030D0000FE915E00E94CD09F80181938F01F5E019
:1030E0000A3B1F07B9F781E06C96E8E00C947D2E4F
:1030F00080914505992787FD9095A92FB92FFC014F
:103100003196EB30F10508F066C0EC5CFF4F0C9493
:103110008E2E62E778E082EE95E00E94982A80E8A1
:1031200093E00E94730C6AE578E082EE95E00E94DD
:10313000982A65E378E082EE95E00E94982A6BE099
:1031400078E082EE95E00E94982A6AEE77E082EEBF
:1031500095E00E94982A6DEB77E082EE95E00E9460
:10316000982A67E977E082EE95E00E94982A63E763
:1031700077E082EE95E00E94982A6CE477E082EE98
:1031800095E00E94982A82EE95E00E94842A0E948F
:10319000A60D21C06FE277E01AC06AE077E017C0A1
:1031A00065EF76E014C066ED76E011C062E976E086
:1031B0000EC06DE776E00BC068E676E082EE95E043
:1031C0000E94982A62E276E002C06CE076E082EE2D
:1031D00095E00E94982A6AE070E080E090E00E940A
:1031E000E12882EE95E00E94BE2B892B29F082EE29
:1031F00095E00E94EB2BF5CF0895ACE1B0E0E3E061
:10320000F9E10C94612E909145059F3F09F023C18F
:10321000482F50E0FA013A97EF36F10508F00FC158
:10322000E15CFF4F0C948E2E61E172E0A0C06DE175
:1032300072E082EE95E00E94AA2A85E789838BE1FD
:10324000EFE9F5E0DE01129601900D928A95E1F723
:103250006CE1CE0101960E941E0C0E949C0B83E043
:103260008093730568EC70E080E090E00E94E128B4
:1032700080917305843009F0E2C08FE70E94BA099B
:103280000E94CD098983853509F0D9C06DEE74E0BF
:1032900082EE95E00E94982A6FEC74E082EE95E051
:1032A0000E94982A61EB74E096C065E372E082EEBA
:1032B00095E00E94AA2A89E6898361E0CE01019601
:1032C0000E941E0C0E949C0B83E08093730568ECA7
:1032D00070E080E090E00E94E128809173058430E6
:1032E00009F0ADC08FE70E94BA090E94CD09898319
:1032F0008E010E5F1F4F7E014DE1E40EF11C0E9416
:10330000CD09F80181938F01EE15FF05C1F78BE11F
:10331000FE013296AFE9B5E001900D928A95E1F792
:103320008981893409F08BC063E974E082EE95E00D
:103330000E94982A65E774E082EE95E00E94982A40
:1033400067E574E048C06FE472E082EE95E00E94A9
:10335000AA2A8EEF8093450572C080528750805311
:1033600090914805981708F066C06EE572E082EE0D
:1033700095E00E94AA2A63C084E18093450560E23B
:1033800074E029C085E18093450569EE73E023C0B0
:1033900086E18093450562EB73E01DC087E1809371
:1033A000450568E673E017C088E18093450567E549
:1033B00073E011C089E18093450563E473E00BC0BD
:1033C0008AE1809345056EE273E005C08BE180934E
:1033D000450566E073E082EE95E00E94982A2FC0D2
:1033E0006CEE72E082EE95E00E94982A8091AD0525
:1033F00091E01DC066ED72E082EE95E00E94982A91
:103400008091AD0592E013C061EC72E082EE95E030
:103410000E94982A8091AD0594E009C066EA72E0A6
:1034200082EE95E00E94982A8091AD0598E0892768
:103430008093AD058FEF809345050E94471082EE83
:1034400095E00E94BE2B892B09F45BC182EE95E0CA
:103450000E94EB2BF4CF0E944611882309F451C13E
:103460008091DF04811104C08FEF8093450541C135
:1034700040E050E060E070E080EE94E00E94052FB4
:1034800040914505042F112707FD1095212F312F5D
:10349000F8013197EB31F10508F01BC1E255FF4F00
:1034A0000C948E2E552747FD50952091480530E00D
:1034B000241735070CF40DC18B019C010150110933
:1034C00021093109003211052105310558F0C0905C
:1034D0004905EBE4F5E0F12CD12CA8E2EA2E4150AD
:1034E00051090FC0FA01E156FA4F61506083D9C00B
:1034F000DF0111972C9130E02417350729F0F39460
:103500003296FC10F5CFCBC00E2D10E020E030E05D
:10351000061717072807390741F42081DA01A15659
:10352000BA4F11962C93DD24D394E394E8CF6F3FE8
:1035300071058105910511F008F0CBC06093B705C6
:10354000B0C06F3F71058105910511F008F0C1C051
:103550006093B805A6C06F3F71058105910511F014
:1035600008F0B7C06093B9059CC02091E0042062C8
:103570002037E9F440E050E060E070E081EE94E054
:103580000E94052F9B01AC01DC01CB010197A10931
:10359000B1090897A105B10508F0AEC0A4EDB0E3EC
:1035A0000E94DF2D6A5E7C4A8A46954E24C02636EC
:1035B000E9F440E050E060E070E081EE94E00E94C9
:1035C000052F9B01AC01DC01CB010197A109B109D9
:1035D0000797A105B10508F08FC0A8EAB1E60E94DF
:1035E000DF2D645E7C438E46944E05C061157105E7
:1035F0008105910579F08B019C010054114E2D49F4
:1036000038410138F0EF1F07FAEF2F07F2E03F07CC
:1036100008F05FC06093AF057093B0058093B1056B
:103620009093B2053EC06F3F71058105910511F081
:1036300008F04FC06093B30534C08B019C0101506A
:103640001109210931090F3F11052105310508F044
:1036500040C06093B40525C08B019C01045C1940F7
:10366000210931090D344DE114072105310528F4F4
:103670007093B6056093B50514C061157105810599
:10368000910521F48FEF8093AE050BC06134710575
:1036900081059105F0F461506093AE0502C0DD2014
:1036A000C1F08091DE0481111AC080917F05909154
:1036B0008005A0918105B09182050196A11DB11DE3
:1036C00080937F0590938005A0938105B093820538
:1036D00006C060E772E082EE95E00E94AA2A0E948E
:1036E0003C118FEF809345056AE082EE95E00E94E1
:1036F000BC2A0E94471005C061E070E080E090E0C5
:103700007ACF6C96E8E00C947D2E6AE572E082EE4A
:1037100095E00E94982A62E472E082EE95E00E94B1
:10372000982A82EE95E00E94BE2B892B31F082EE22
:1037300095E00E94EB2B0E94FD180E94D517823065
:1037400029F0833051F46DE072E002C064E272E06F
:1037500082EE95E00E94982A08958FEF80934505A8
:103760001092DE040E944710809145058E3F69F05B
:1037700082EE95E00E94BE2B892BB1F382EE95E09C
:103780000E94EB2B0E94FD18EFCF08950F931F931B
:10379000109145051F3F09F0D2C0893409F457C084
:1037A00000F5883309F469C058F4803309F477C010
:1037B00008F061C08B3109F440C08132B1F1B9C069
:1037C000813409F487C030F4893309F466C0803449
:1037D00061F1AFC0823409F48EC0863409F448C068
:1037E000A8C0823609F487C078F4883531F128F40E
:1037F0008235C1F18335E1F09CC08A3509F494C06B
:10380000813609F467C095C0823761F128F48636A5
:1038100079F18936E1F08DC0883779F08A3709F47B
:1038200083C0833709F085C003C061E172E015C031
:103830000E94770D6EE872E004C00E94800D68EA75
:1038400072E082EE95E00E94AA2A8EEF70C00E947C
:103850007A060E94BF0667EC72E082EE95E00E9455
:10386000AA2A67C081E00E94DF0660EE72E0F5CF11
:103870000E94F1105EC080535AC06AEF71E082EE80
:1038800095E00E94982A90919E0588E0890F8871A2
:10389000977E892B80939E051AC089E048C067EE09
:1038A00071E082EE95E00E94982A8091BF05909188
:1038B000C005A091C105B091C20520E18227809387
:1038C000BF059093C005A093C105B093C2051093A6
:1038D00045052FC061ED71E082EE95E00E94982AC7
:1038E0008091BF059091C005A091C105B091C2051E
:1038F00040E4842710C060EC71E082EE95E00E9405
:10390000982A8091BF059091C005A091C105B09102
:10391000C20520E282278093BF059093C005A09343
:10392000C105B093C20502C00E94851B8FEF809332
:103930004505809145058E3F09F0D4C0DDC00E9449
:103940004611882309F4D8C08091DF04811104C096
:103950008FEF80934505C6C040E050E060E070E026
:1039600080EE94E00E94052F00914505112707FD88
:103970001095212F312FF8013197E930F10508F02A
:10398000B4C0E753FF4F0C948E2E8B019C01015461
:10399000114E2D4938410F37104F2A4F324008F051
:1039A000A4C060937B0570937C0580937D05909304
:1039B0007E0577C060937F057093800580938105B5
:1039C0009093820581E08093DE046BC068307105BE
:1039D0008105910508F089C06093830562C08B0161
:1039E0009C0101501109210931090A3011052105F5
:1039F000310508F07AC06093840553C061EB71E033
:103A000080EE94E00E943F3010E0009799F00E9411
:103A10001930009779F0183130F4E12FF0E0EA58CE
:103A2000FA4F87871F5F61EB71E080E090E00E94B2
:103A30003F30EBCF1831A8F5E12FF0E0EA58FA4F0C
:103A400017861F5FF7CF653071058105910508F076
:103A50004CC060939D0525C08B019C01015011094C
:103A6000210931090630110521053105F0F52091B4
:103A70009E05287F262B20939E0513C08B019C0159
:103A800001501109210931090115124C214031055C
:103A900060F560937705709378058093790590932E
:103AA0007A058091DE04811113C080917F05909189
:103AB0008005A0918105B09182050196A11DB11DDF
:103AC00080937F0590938005A0938105B093820534
:103AD0000E943C118FEF809345056AE082EE95E0ED
:103AE0000E94BC2A0E94781807C060E772E082EE4C
:103AF00095E00E94AA2AECCF1F910F9108958FEFB5
:103B0000809345051092DE040E9478188091450547
:103B10008E3F69F082EE95E00E94BE2B892BB1F3B7
:103B200082EE95E00E94EB2B0E94C61BEFCF6AE06D
:103B300070E080E090E00E94E12882EE95E00E9433
:103B4000BE2B892B29F082EE95E00E94EB2BF5CF5E
:103B50000895CF93C82F682F82EE95E00E94182C0D
:103B600090916A059C2790936A05CF910895A1E0F2
:103B7000B0E0EDEBFDE10C94672E99830E94A91D46
:103B80009981892F0E94A91D2196E2E00C94832E31
:103B90001F93CF93DF93182FEB0110926A0565EB0B
:103BA00070E082EE95E00E94590662E670E082EED7
:103BB00095E00E945906812F0E94A91DCE010E9406
:103BC000B71DDF91CF911F91089560916A0582EE34
:103BD00095E00E94182C0895A1E2B0E0E2EFFDE12B
:103BE0000C94632E7B018A018C3009F452C108F0D9
:103BF00040C0863009F4BCC018F5833009F491C088
:103C000070F4813009F472C0823009F047C26BE170
:103C100070E082E00E94C81D0FE915E078C0843092
:103C200009F487C0853009F039C26091490570E018
:103C3000660F771F85E00E94C81D0AE415E086C064
:103C4000893009F4A7C070F4873009F49BC088302C
:103C500009F024C261E070E088E00E94C81D8091F4
:103C6000D40522C28A3009F4CAC08B3009F4F1C0ED
:103C700015C28A3609F474C1D8F4873609F439C1FB
:103C800038F4853609F40DC1863609F41EC106C222
:103C9000883609F436C1893609F000C261E070E067
:103CA00089E60E94C81D0E947A060E94BF06F4C1E0
:103CB0008D3609F4D3C138F48B3609F490C18C36B3
:103CC00009F499C1EBC18E3609F4DBC1873C09F0D8
:103CD000E5C161E070E087EC0E94C81D81E00E94B0
:103CE000A91D0E94E51D10926B05E2C169E270E01A
:103CF00081E00E94C81D06E715E0F80181918F015F
:103D00000E94A91DF5E00F391F07B9F7CFC1F801CF
:103D100081918F010E94A91DF5E00A3B1F07B9F7A9
:103D2000C5C161E070E083E00E94C81D0E94D51704
:103D3000BBC161E070E084E00E94C81D81E00E9488
:103D4000A91D0E94E51D0E940816B2C18091490577
:103D500090E0880F991F98012A5435402817390799
:103D600008F0A4C1F80181918F010E94A91DEECF36
:103D700062E070E086E00E94C81D80E893E00E9447
:103D8000B71D94C161E070E087E00E94C81D80917A
:103D900048058AC186E6898361E0CE0101960E94CA
:103DA0001E0C0E949C0B83E08093730568EC70E00E
:103DB00080E090E00E94E128809173058430D9F47E
:103DC0008FE70E94BA090E94CD098983863469F47D
:103DD00060E270E089E00E94C81D10E20E94CD09F7
:103DE0000E94A91D1150D1F761C161E070E089E026
:103DF0000E94C81D51C161E070E089E052C169E1D3
:103E000070E08AE00E94C81D1092BA0520917205E8
:103E10008091BF059091C005A091C105B091C205E8
:103E2000222311F0806801C08F778093BF059093A3
:103E3000C005A093C105B093C2050AEB15E0F801D7
:103E400081918F010E94A91DF5E0033D1F07B9F77D
:103E50002DC161E270E08BE00E94C81D8091AA0430
:103E60008F3F39F08091AA0491E0980F9093AA04B3
:103E700002C08091AA040E94A91D10E0812F0E9417
:103E8000EA150E944C090E94B71D1F5F1031B1F75F
:103E90000DC161E070E08CE00E94C81D8091D305E7
:103EA00003C161E070E085E60E94C81D89E2E81662
:103EB000F10409F0F8C0D801E6E7F5E08D918193AF
:103EC00085E0EF39F807D1F7E7C061E070E086E6FA
:103ED0000E94C81DEBE1EE16F10409F0E4C0D80120
:103EE000EFE9F5E08D91819385E0EA3BF807D1F7A2
:103EF000D3C061E070E087E60E94C81D0E94770D84
:103F0000CBC061E070E088E60E94C81D85E7898328
:103F10008BE1EFE9F5E0DE01129601900D928A95B2
:103F2000E1F76CE1CE0101960E941E0C0E949C0BF1
:103F300083E08093730560E273E080E090E00E948C
:103F4000E12880917305843009F0ADC08FE70E94AD
:103F5000BA090E94CD098983853509F0A4C09CC0A7
:103F600061E070E08AE60E94C81D89E6898361E00D
:103F7000CE0101960E941E0C0E949C0B83E0809350
:103F8000730560E273E080E090E00E94E128809198
:103F90007305843009F087C08FE70E94BA090E9438
:103FA000CD0989838E010E5F1F4F7E01EDE1EE0E7C
:103FB000F11C0E94CD09F80181938F01EE15FF05D8
:103FC000C1F78BE1FE013296AFE9B5E001900D92A9
:103FD0008A95E1F78981893409F065C05DC061E0A7
:103FE00070E08BE60E94C81DF80180818093D405A3
:103FF0000E94800D51C061E070E08CE60E94C81DF7
:10400000F0E2EF16F10461F487E6898380E2F801BB
:10401000DE01129601900D928A95E1F761E203C0EC
:1040200087E4898361E0CE0101960E941E0C0E9404
:104030009C0B83E0809373056CE474E080E090E077
:104040000E94E12880917305843069F58FE70E9412
:10405000BA090E94CD09873431F51EC061E070E0D5
:104060008DE60E94C81D89E1E816F104E1F4D8014B
:10407000EAEBF5E08D91819385E0E33DF807D1F718
:104080000BC061E070E08EE60E94C81DF8018081DF
:104090008093D3050E94600D81E006C061E070E06E
:1040A0008AEC0E94C81D80E00E94A91D0E94E51DA7
:1040B000A196E6E00C947F2EA0E0B0E0E2E6F0E20C
:1040C0000C94612ECAECD3E014E606E035E0F32E42
:1040D00044E0E42E53E0D52E62E0C62E82EE95E059
:1040E0000E94BE2B892B09F49BC082EE95E00E94B2
:1040F000EB2B282F809335044091340450E0473057
:10410000510560F7FA01EE52FF4F0C948E2E853B5D
:1041100029F781E080933404E1CF823609F07DC035
:10412000C0923404DBCF8093330480933204D09266
:104130003404D4CF9C0133273093310420933004CE
:1041400090913204982790933204E0923404C6CFC1
:10415000382F22274091300450913104242B352BE5
:104160003093310420933004909132049827909337
:104170003204F09234042536310508F4AFCF61E003
:1041800070E08CEC0E94C81D81E00E94A91D0E9475
:10419000E51D43C020912E0430912F04F901E65310
:1041A000FC4F808390913204982790933204C90188
:1041B000019690932F0480932E0420913004309127
:1041C00031048217930708F489CF0093340486CF13
:1041D0008091320482130BC060912E0470912F04E1
:1041E0004AEC53E0809133040E94EC1D0DC062E064
:1041F00070E08BEC0E94C81D809133040E94A91DC1
:1042000080916A050E94A91DFE01812F11928A9555
:10421000E9F710922F0410922E04109234045ECF0E
:10422000CDB7DEB7E8E00C947D2E81E080936B057E
:1042300080916B05882349F082EE95E00E94BE2BA9
:10424000892BB1F30E945C20F3CF0895AAE2B0E07D
:10425000ECE2F1E20C945F2E0E94B2286B017C012B
:1042600081E00E94C10A82EE95E00E94BE2B892B5C
:1042700029F082EE95E00E94EB2BF5CF5E984098F6
:1042800011E072E6B72EE9E2AE2E03E00E94B228FA
:104290006C197D098E099F09693C7105810591059D
:1042A000E0F11123D1F10E94B2286B017C015D9AEB
:1042B000419A80ED97E00E94B607B982E6E7F5E003
:1042C000DE0112968A2D01900D928A95E1F76AE23D
:1042D000CE0101960E941E0C5D98419880E090E00E
:1042E0000E94B607009373050E949C0B62E370E086
:1042F00080E090E00E94E12880917305843061F4B1
:10430000009373058FE70E94BA090E94CD0911E05E
:10431000823419F410E001C011E082E10E94D72933
:10432000892BA1F411E012C05E9A409A5D9A419ADD
:1043300082EE95E00E94EB2B8D309105B9F06CF484
:104340000A97A1F05E9840985D98419882EE95E0BA
:104350000E94BE2B892B41F799CF8332910579F0CA
:104360008234910579F70E941521ECCF62EB71E060
:1043700082EE95E00E94982A0E947F1DE3CF0E9462
:104380000816E0CF8F929F92AF92BF92CF92DF92AA
:10439000EF92FF921F93CF93DF9382E10E94D72980
:1043A000892B09F089C068EC70E080E090E00E9401
:1043B000E12880E090E00E94B6070E94B2284B01FD
:1043C0005C016B017C0180ECC80E82E1D81EE11C0F
:1043D000F11C0E94B2286C157D058E059F0530F4F6
:1043E00082E10E94D729892BA1F364C082E10E9457
:1043F000D729892B09F05EC080ED97E00E94B607AF
:104400000E94B2286B017C01D0E0C1E088E4880EF4
:1044100086E2981EA11CB11C11E082E10E94D729FE
:10442000892B21F58C149D04AE04BF0430F480ED7B
:1044300097E00E94B607D1E0F0CF0E94B2286C1935
:104440007D098E099F09693C71058105910528F355
:104450000E94B2286B017C01C12719F080ED97E022
:1044600002C080E090E00E94B607D7CF80E090E0E5
:104470000E94B607DD23B9F08091D30590E0019644
:1044800065E070E00E94022E8093D3050E94600DCB
:104490000E94DF130E94800D64EF71E080E090E0E5
:1044A0000E94E12809C080E00E94DF060E94F81106
:1044B0000E94770D0E942621DF91CF911F91FF90DE
:1044C000EF90DF90CF90BF90AF909F908F90089526
:1044D000CF92DF92EF92FF9280E00E941D080E942F
:1044E000F40761E086E00E946B2961E085E00E94AC
:1044F0006B2961E08EE00E946B2961E08FE00E94F1
:104500006B2960E082E10E946B2960E088E00E94F4
:104510006B2961E088E00E94A4290E949F0740E087
:1045200052EC61E070E082EE95E00E94062D0E9460
:10453000DF130E94800D0E94C4138FEF8093AA04A2
:104540000E94090878940E94B2286B017C01809136
:10455000AA048F3F59F40E94B2286C197D098E0974
:104560009F09603D77408105910588F380ED97E0D4
:104570000E94B60761E082E10E94A4295E9A409AF7
:1045800082EE95E00E94BE2B892B29F082EE95E009
:104590000E94EB2BF5CF6DEF72E082EE95E00E946A
:1045A000792A80E893E00E94730C64E173E082EE64
:1045B00095E00E94792A4AE050E065E070E082EEE2
:1045C00095E00E94492B62E370E080E090E00E9459
:1045D000E12882EE95E00E94BE2B04970CF182EE5A
:1045E00095E00E94EB2B82349105D1F482EE95E0A8
:1045F0000E94EB2B8E34910599F482EE95E00E9497
:10460000EB2B8434910561F482EE95E00E94EB2B54
:10461000819731F480E090E00E94B6070E94262145
:1046200040917705509178056091790570917A05F0
:10463000DB01CA010197A109B1090497A105B105E0
:1046400068F44093A904433029F440EA56E861E055
:1046500070E004C040E052EC61E070E082EE95E072
:104660000E94062D0E94C2215E98409880E090E052
:104670000E94B6070E94C4131092C5048091BF0522
:1046800083FF11C080918B05882351F080919205A2
:10469000882331F080919905882311F087E001C0CB
:1046A00085E08093C50480E00E94C10A8091C60421
:1046B0000E94F5090E949C0B10923F0410923E0448
:1046C00010923D04F12C8091D4058F15B0F062E377
:1046D00070E080E090E00E94E12880ED97E00E9489
:1046E000B60762E370E080E090E00E94E12880E09D
:1046F00090E00E94B607F394E6CF80919E0584FF78
:1047000008C0982F987181E0983109F080E00E94EC
:10471000B4118FE00E941D08FF90EF90DF90CF90C2
:104720000895EF92FF920F931F93CF93DF938C0125
:104730006EE770E082EE95E00E945906E801F12CE8
:10474000F0E2EF2E8E0188818D57823048F46DE7BC
:1047500070E082EE95E00E94590688818E2588835C
:104760002196F801608182EE95E00E94182CF39466
:10477000F9E0FF12E7CF6EE770E082EE95E00E946D
:104780005906CDB7DEB7E6E00C947F2EA9E0B0E085
:10479000ECECF3E20C94672E9091C70491110EC0DB
:1047A0009EEF99838A836B8350E0559547954C83A0
:1047B0002D83198618861F821E822EC04091CC043C
:1047C000842F90E0B4E095958795BA95E1F7242F72
:1047D0002F7030E08217930719F18DEF89831B82C8
:1047E000FE01349650E0842F90E0A4E095958795E3
:1047F000AA95E1F7242F2F7030E08217930749F034
:10480000DC01A353BB4F8C918193405F5F5F5630B7
:1048100051F74093CC045A83CE0101960E94912314
:104820008091C70490E0019666E070E00E94022E3D
:104830008093C7042996E2E00C94832EA0E0B0E0B8
:10484000E4E2F4E20C94602E6C016EE770E082EE1C
:1048500095E00E9459068601E12CF12CC0E0D0E0E1
:1048600030E2B32EF801608183E8860F823078F45D
:104870006DE770E082EE95E00E945906F8016081D4
:104880006B2570E082EE95E00E94590604C082EE2E
:1048900095E00E94182CE114F10459F0F801808190
:1048A0009E01280F311DC901C92FDD27C80FD91F4F
:1048B000DD273FEFE31AF30A89E0E816F10459F027
:1048C00028E0E216F10421F48C2F8095F601808710
:1048D0000F5F1F4FC7CFCDB7DEB7E9E00C947C2E3A
:1048E000A9E0B0E0E6E7F4E20C94672EE82F362F5B
:1048F0008091C70490E0019664E270E00E94022E6D
:104900008093C70458E9598350E15A83813089F074
:1049100048F08230B9F08330D9F48B8381EF8C83F7
:104920003D8319C085E08B8381EF8C832F5F2D83BE
:1049300012C08B8381EF8C8384E6489FA0011124F1
:104940005D8309C084E08B8381EF8C83ED8303C09A
:104950000E94F11104C0CE0101960E941E242996E6
:10496000E2E00C94832EA2E0B0E0E9EBF4E20C94D8
:104970005C2E182F762E2A8349830E94BE286B0155
:104980007C018091DD048090C8049090C904A090BF
:10499000CA04B090CB042A8149818823C1F0D70191
:1049A000C60188199909AA09BB094C015D0191EE5C
:1049B00089169EE29906A104B10420F1241708F497
:1049C000422F202F672D812F0E94702413C0D70102
:1049D000C60188199909AA09BB094C015D0191E337
:1049E000891695E79906A104B10460F0672D812F1F
:1049F0000E94C623C092C804D092C904E092CA049F
:104A0000F092CB042296EDE00C94782EA2E2B0E076
:104A1000ECE0F5E20C945D2E8CE00E94DC09811143
:104A20000FC06CE173E082EE95E00E94AA2A5E9AC4
:104A3000409A80E00E94C10A0E949C0B5E984098B8
:104A400082EE95E00E94BE2B892B01F182EE95E06B
:104A50000E94EB2B9091A904992319F00E94F21364
:104A6000EFCF40913E0450E09A012F5F3F4F2F71EE
:104A7000332760913F0470E02617370709F3FA01E6
:104A8000E75BFB4F808320933E04DACF8091730570
:104A9000843009F086C00E94BE2861157105810529
:104AA000910549F06093B7047093B8048093B904FA
:104AB0009093BA040CC081E090E0A0E0B0E0809355
:104AC000B7049093B804A093B904B093BA0480914A
:104AD000AD049091AE0481609093AE048093AD04D8
:104AE00083E0809373058FE70E94BA0909E614E01A
:104AF0000E94CD09F80181938F01F4E002371F076E
:104B0000B9F72091720480916904982F922796FF3B
:104B10003BC090E4922790937204982F9873983337
:104B2000F1F410E0212F30E080916904877090E06B
:104B3000821793074CF11F5F20919E05812F90E013
:104B4000FC01E759FB4F24FF04C080810E94D31170
:104B5000E9CF608182EE95E00E94182CE3CF8F733D
:104B600099F480916A048093B60480916B048093D9
:104B7000B40480916C048093B30480916F0490E03E
:104B80009093AC048093AB0480913D04813019F480
:104B900082E080933D0480913D04833011F41092B3
:104BA0003D040E94BE286B017C018091AF0490916E
:104BB000B004A091B104B091B2040097A105B10571
:104BC000C9F0A7019601281B390B4A0B5B0BDA01D0
:104BD000C901883B9B40A105B10560F00E940B0A0A
:104BE0008093B5041092AF041092B0041092B104F7
:104BF0001092B2048091BB049091BC04A091BD04BA
:104C0000B091BE0446015701881A990AAA0ABB0A44
:104C100086E795E00E94370886169706A806B9062B
:104C200008F4A9C0C092BB04D092BC04E092BD04B9
:104C3000F092BE040E9457068091AA048830A0F02A
:104C40008091BF059091C005A091C105B091C205AA
:104C50006CE1B695A795979587956A95D1F7892BBD
:104C60008A2B8B2B09F0A8C18091AA048F5F8093B7
:104C7000AA048091B7049091B804A091B904B091AE
:104C8000BA040097A105B105F1F0C81AD90AEA0AD9
:104C9000FB0A86E795E00E9437086C157D058E05B6
:104CA0009F0508F008C18091BF0584FD04C080ED18
:104CB00097E00E94B6071092B7041092B8041092C1
:104CC000B9041092BA0490917204907C909372048B
:104CD00050913E0480913F0420913D04581709F4FF
:104CE00007C1223009F004C1905890937204E091FA
:104CF0009E05E770F0E0E658FC4F6081693008F0EF
:104D0000DFC0615040E04613DDC080933F0487E37D
:104D1000840F90917204892B809372044093400415
:104D200083E080933D045D9A419A80918305909140
:104D3000C504911132C10E94BC0A8091C6040E9430
:104D4000F509E0919E05E770F0E0E658FC4F6081C0
:104D500082E794E00E94D70BE091C604EF5FE093F6
:104D6000C604E83109F425C1F0E0EA58FA4F878516
:104D7000882309F41EC10E94460C813069F5809198
:104D80009E05887149F18091AD049091AE04880F21
:104D9000991F9093AE048093AD0483E080937305D4
:104DA0000E949C0B0E94BE286093AF047093B004D5
:104DB0008093B1049093B204672B682B692B61F444
:104DC00081E090E0A0E0B0E08093AF049093B00465
:104DD000A093B104B093B20480919E0584FF1FC0DC
:104DE0008091AD049091AE048E7F0E946D09182FC2
:104DF0006091AB048091B6040E94E813482F612FA4
:104E00008091B50449A30E94E8130091D405282F8E
:104E100049A16091B3048091B4040E94B3245D98C9
:104E200041988091C3048130C1F018F08230B1F113
:104E3000D1C082E10E94D729892B09F0CBC081E043
:104E40008093C3040E94B2286093BF047093C0048F
:104E50008093C1049093C204BDC082E10E94D7290F
:104E6000892B31F50E94B228C090BF04D090C004B5
:104E7000E090C104F090C2046C197D098E099F096D
:104E8000693E73408105910508F4A4C082E08093D7
:104E9000C30480ED97E00E94B6079CC082E10E94A7
:104EA000D729892B09F496C080E090E00E94B607CC
:104EB0001092C3048FC080E090E00E94B60703CF39
:104EC00068E020CF851709F420CF4F5F242F30E012
:104ED00090E0F901EE58FB4FDC01A75BBB4F7C91E2
:104EE0007083F901E05CFB4F708301968F710BCFEB
:104EF0002430B1F42091400481E494E0A3E7B4E0CD
:104F0000FC013E2F381B321718F431913D93F9CF35
:104F100087E3820F90917204892B8093720400CFF3
:104F20008091C304823071F49160909372045E9A10
:104F3000409A53ECE52E55E0F52E8E010F5F1F4F82
:104F4000B80111C05E98409880913D04811103C062
:104F500081E080933D0480913D04833051F784E0EB
:104F600080933D04E6CFF70181917F0169A37AA385
:104F70000E94EA15F801819391938F0169A17AA1AA
:104F8000F3EDEF16F5E0FF0671F780919E0543E71C
:104F900054E087700E94BC08C6CE882309F4CBCEAB
:104FA0002091C40431E0320F3093C4042913C3CEDE
:104FB0000DC01092C604DFCE8091AA04883011F48F
:104FC0005E9A409A89E08093AA04D5CE1092C404D8
:104FD0008150B1CEA296ECE00C94792E8230E8F4A8
:104FE000E82FF0E0EE0FFF1FEB52FA4F7183608362
:104FF000813041F0809169008C7F842B809369001F
:10500000E89A089580916900440F551F440F551F79
:10501000837F842B80936900E99A08951F920F92F1
:105020000FB60F9211242F933F934F935F936F937B
:105030007F938F939F93AF93BF93EF93FF93809151
:10504000D5059091D605892B29F0E091D505F091F1
:10505000D6050995FF91EF91BF91AF919F918F91E7
:105060007F916F915F914F913F912F910F900FBE64
:105070000F901F9018951F920F920FB60F92112448
:105080002F933F934F935F936F937F938F939F9350
:10509000AF93BF93EF93FF938091D7059091D8057D
:1050A000892B29F0E091D705F091D8050995FF915A
:1050B000EF91BF91AF919F918F917F916F915F9190
:1050C0004F913F912F910F900FBE0F901F90189509
:1050D0001F920F920FB60F9211242F933F938F932D
:1050E0009F93AF93BF938091DA059091DB05A091D8
:1050F000DC05B091DD053091D90523E0230F2D3774
:1051000020F40196A11DB11D05C026E8230F0296CB
:10511000A11DB11D2093D9058093DA059093DB057D
:10512000A093DC05B093DD058091DE059091DF054D
:10513000A091E005B091E1050196A11DB11D8093FC
:10514000DE059093DF05A093E005B093E105BF91E4
:10515000AF919F918F913F912F910F900FBE0F9024
:105160001F9018952FB7F8946091DA057091DB05C0
:105170008091DC059091DD052FBF08953FB7F8942D
:105180008091DE059091DF05A091E005B091E105E9
:1051900026B5A89B05C02F3F19F00196A11DB11D92
:1051A0003FBF6627782F892F9A2F620F711D811DAF
:1051B000911D42E0660F771F881F991F4A95D1F70E
:1051C0000895CF92DF92EF92FF92CF93DF936B011E
:1051D0007C010E94BE28EB01C114D104E104F1045A
:1051E00079F00E94BE286C1B7D0B683E7340A0F3D3
:1051F00081E0C81AD108E108F108C851DC4FECCFB2
:10520000DF91CF91FF90EF90DF90CF900895789449
:1052100084B5826084BD84B5816084BD85B58260BB
:1052200085BD85B5816085BDEEE6F0E08081816059
:105230008083E1E8F0E01082808182608083808159
:1052400081608083E0E8F0E0808181608083E1EB31
:10525000F0E0808184608083E0EBF0E08081816019
:105260008083EAE7F0E080818460808380818260CF
:1052700080838081816080838081806880831092B8
:10528000C1000895833081F028F4813099F0823094
:10529000A1F008958630A9F08730B9F08430D1F4B8
:1052A000809180008F7D03C0809180008F778093F4
:1052B0008000089584B58F7702C084B58F7D84BD4A
:1052C00008958091B0008F7703C08091B0008F7DEA
:1052D0008093B0000895CF93DF9390E0FC01ED50F0
:1052E000F44F2491FC01E95FF34F8491882349F145
:1052F00090E0880F991FFC01E15DF34FA591B491F7
:105300008B5D934FFC01C591D4919FB7611108C08B
:10531000F8948C91209582238C93888182230AC0F3
:10532000623051F4F8948C91322F309583238C9312
:105330008881822B888304C0F8948C91822B8C9373
:105340009FBFDF91CF910895A1E0B0E0EAEAF9E2D2
:105350000C94652E282F30E0F901E152F44F84912E
:10536000F901ED50F44F1491F901E95FF34F049105
:105370000023C9F0882321F069830E9442296981B2
:10538000E02FF0E0EE0FFF1FEB5DF34FA591B4911E
:105390009FB7F8948C91611103C01095812301C0CF
:1053A000812B8C939FBF2196E4E00C94812ECF93A8
:1053B000DF93282F30E0F901E152F44F8491F90195
:1053C000ED50F44FD491F901E95FF34FC491CC2330
:1053D00091F081110E944229EC2FF0E0EE0FFF1FA7
:1053E000E55EF34FA591B4912C912D2381E090E0DF
:1053F00021F480E002C080E090E0DF91CF91089539
:105400008E3008F08E50877020919D0190E4299F86
:1054100090011124822B80937C0080917A0080641B
:1054200080937A0080917A0086FDFCCF809178008D
:105430002091790090E0922B0895A0E0B0E0E3E2A3
:10544000FAE20C94612E6C017A01EB01E60EF71E74
:1054500000E010E0CE15DF0561F06991D601ED9115
:10546000FC910190F081E02DC6010995080F191FEC
:10547000F1CFC801CDB7DEB7E8E00C947D2E611501
:10548000710589F0DB010D900020E9F7AD01415075
:105490005109461B570BDC01ED91FC910280F38111
:1054A000E02D0995089580E090E00895EF92FF9235
:1054B0000F931F93CF93DF938C01FB01C0E0D0E0EB
:1054C00064917F018FEFE81AF80A662361F0D80132
:1054D000ED91FC910190F081E02DC8010995C80F74
:1054E000D91FF701EDCFCE01CDB7DEB7E6E00C94C2
:1054F0007F2E0E943F2A0895DC01ED91FC910190DE
:10550000F081E02D099508950F931F93CF93DF93BA
:10551000EC016DE00E947C2A8C016AE0CE010E94C1
:105520007C2A800F911FDF91CF911F910F910895D9
:105530000F931F93CF93DF93EC010E94562A8C01A7
:10554000CE010E94842A800F911FDF91CF911F917D
:105550000F9108950F931F93CF93DF93EC010E9457
:105560003F2A8C01CE010E94842A800F911FDF9177
:10557000CF911F910F9108950F931F93CF93DF93B6
:10558000EC010E947C2A8C01CE010E94842A800FAB
:10559000911FDF91CF911F910F910895A1E2B0E08B
:1055A000E4EDFAE20C945D2E7C01C42EE52FCB01D4
:1055B000D22E19A221E02D1510F02AE0D22E8E0154
:1055C0000F5D1F4F8D2C912CA12CB12C6C2D7E2F9B
:1055D000A50194010E94162E8C2DD29E80191124B3
:1055E000015011098A3010F4805D01C0895CF80116
:1055F0008083211531054105510521F0C22EE32F8D
:10560000CA01E4CFB801C7010E943F2AA196ECE08D
:105610000C94792EA0E0B0E0E0E1FBE20C94612E66
:10562000EC016A017B012115310541F4E881F98122
:105630000190F081E02D642F09951DC02A303105BD
:10564000A9F477FF12C06DE20E947C2A8C014427E6
:105650005527BA014C195D096E097F092AE0CE0170
:105660000E94CE2A800F911F06C02AE0B701A60132
:10567000CE010E94CE2ACDB7DEB7E8E00C947D2E95
:105680009A01AB01662757FD6095762F0E940A2B81
:1056900008950F931F93CF93DF93EC019A01AB0111
:1056A000662757FD6095762F0E940A2B8C01CE014C
:1056B0000E94842A800F911FDF91CF911F910F913B
:1056C00008952115310549F4DC01ED91FC9101901B
:1056D000F081E02D642F099508950E94CE2A089547
:1056E0009A01462F50E060E070E00E94612B08951F
:1056F0009A01AB0160E070E00E94612B08950F9366
:105700001F93CF93DF93EC010E94612B8C01CE019C
:105710000E94842A800F911FDF91CF911F910F91DA
:1057200008950F931F93CF93DF93EC019A01AB0180
:1057300060E070E00E94612B8C01CE010E94842AFF
:10574000800F911FDF91CF911F910F9108950F93BB
:105750001F93CF93DF93EC019A01462F50E060E056
:1057600070E00E94612B8C01CE010E94842A800F80
:10577000911FDF91CF911F910F910895FC01248516
:105780003585F901E05CFF4F80819181F901EE5B85
:10579000FF4F20813181821B930B8F7399270895CE
:1057A000FC0184859585FC01E05CFF4F40815181BF
:1057B000FC01EE5BFF4F208131814217530741F01E
:1057C0000190F081E02DE80FF91F808190E00895AD
:1057D0008FEF9FEF0895FC0184859585FC01E05CC7
:1057E000FF4F40815181FC01EE5BFF4F20813181F1
:1057F0004217530779F0A081B181A80FB91F8C918E
:10580000208131812F5F3F4F2F73332731832083D6
:1058100090E008958FEF9FEF0895FC0181A1882308
:1058200029F0A489B5898C9186FFFBCF11A2089538
:10583000CF93DF93FC0126853785D901A05CBF4F4C
:105840008D919C91119701968F739927E901CE5BF9
:10585000DF4F4881598184179507D9F30D90BC918A
:10586000A02DA20FB31F6C93A685B785A05CBF4F78
:1058700011969C938E93A689B7892C9181E090E034
:10588000078C02C0880F991F0A94E2F7282B2C93EB
:1058900081E081A30488F589E02D80818064808384
:1058A00081E090E0DF91CF91089508951F920F92CB
:1058B0000FB60F9211242F933F934F938F939F9383
:1058C000EF93FF938091C00082FD1CC04091C60001
:1058D000809188069091890601968F73992720916F
:1058E0008A0630918B068217930771F0E091880643
:1058F000F0918906E85BF94F408390938906809385
:10590000880602C08091C600FF91EF919F918F9110
:105910004F913F912F910F900FBE0F901F901895B0
:1059200082EE95E00E94BE2B892B11F00E94552C2F
:1059300008951F920F920FB60F9211242F933F9349
:105940008F939F93EF93FF932091440630914506E8
:1059500080914606909147062817390731F48091C7
:10596000C1008F7D8093C10014C0E0914606F09184
:105970004706EC5FF94F20818091460690914706DB
:1059800001968F739927909347068093460620933C
:10599000C600FF91EF919F918F913F912F910F90B2
:1059A0000FBE0F901F901895A0E0B0E0EAEDFCE26A
:1059B0000C945D2EFC011382128288EE93E0A0E02D
:1059C000B0E084839583A683B7838CEB93E09183C7
:1059D00080837587648757874687318B208B138B2D
:1059E000028BF58AE48AD78AC68AB18EA08E938EFE
:1059F000828E8F85848F8889858F8989868F8A8911
:105A0000878F8B8980A3ECE00C94792ECF92DF9264
:105A1000EF92FF92CF93DF93EC016A017B01411576
:105A200081EE580761057105F9F0EC89FD8981E087
:105A300090E008A002C0880F991F0A94E2F78083C3
:105A400060E079E08DE390E0A70196010E94162EB8
:105A500021503109410951095695479537952795A8
:105A6000211580E1380798F0EC89FD89108260E803
:105A700074E88EE190E0A70196010E94162E215055
:105A80003109410951095695479537952795E88978
:105A9000F9893083EA89FB89208319A2EE89FF897D
:105AA000408181E090E09C010C8C02C0220F331FEA
:105AB0000A94E2F7422B4083EE89FF8940819C01E2
:105AC0000D8C02C0220F331F0A94E2F7422B408351
:105AD000EE89FF8940819C010E8C02C0220F331F8A
:105AE0000A94E2F7422B4083EE89FF8920810F8CD4
:105AF00002C0880F991F0A94E2F780958223808361
:105B0000DF91CF91FF90EF90DF90CF9008958F922B
:105B10009F92AF92BF92CF92DF92EF92FF920F933C
:105B20001F9381E08F9385E08F9387E08F9383E0CD
:105B30008F9384E08F93E6EC8E2E912CF2ECAF2EB7
:105B4000B12CA1ECCA2ED12CB0ECEB2EF12C04EC34
:105B500010E025EC30E044E056E068E476E082EEC8
:105B600095E00E94D42C0F900F900F900F900F9003
:105B70001F910F91FF90EF90DF90CF90BF90AF906B
:105B80009F908F9008950E9407290E946822C0E983
:105B9000DCE20E9406252097E1F30E94902CF9CFC9
:105BA000A29FB001B39FC001A39F700D811D11245E
:105BB000911DB29F700D811D1124911D08950E94A9
:105BC000D02DA59F900DB49F900DA49F800D911D89
:105BD00011240895B7FF0C94DF2D0E94DF2D821B46
:105BE000930B0895DB018F939F930E94DF2DBF914C
:105BF000AF91A29F800D911DA39F900DB29F900D1C
:105C00001124089597FB072E16F4009407D077FD12
:105C100009D00E94942E07FC05D03EF49095819502
:105C20009F4F0895709561957F4F0895A1E21A2EB8
:105C3000AA1BBB1BFD010DC0AA1FBB1FEE1FFF1F30
:105C4000A217B307E407F50720F0A21BB30BE40B80
:105C5000F50B661F771F881F991F1A9469F76095C7
:105C60007095809590959B01AC01BD01CF01089581
:105C7000052E97FB1EF400940E944F2E57FD07D06F
:105C80000E94162E07FC03D04EF40C944F2E509514
:105C90004095309521953F4F4F4F5F4F0895909518
:105CA0008095709561957F4F8F4F9F4F08952F92EC
:105CB0003F924F925F926F927F928F929F92AF929C
:105CC000BF92CF92DF92EF92FF920F931F93CF93E9
:105CD000DF93CDB7DEB7CA1BDB0B0FB6F894DEBF80
:105CE0000FBECDBF09942A88398848885F846E84A6
:105CF0007D848C849B84AA84B984C884DF80EE80F0
:105D0000FD800C811B81AA81B981CE0FD11D0FB6F8
:105D1000F894DEBF0FBECDBFED010895EE0FFF1F5B
:105D20000590F491E02D0994AA1BBB1B51E107C01B
:105D3000AA1FBB1FA617B70710F0A61BB70B881F1B
:105D4000991F5A95A9F780959095BC01CD010895AA
:105D50008F929F92AF92BF92CF92DF92EF92FF927B
:105D6000CF93DF93EC01688179818A819B816115F2
:105D700071058105910521F464E279ED8BE597E0E9
:105D80002DE133EF41E050E00E94382E49015A01E5
:105D90009B01AC01A7EAB1E40E94DF2D6B017C01FD
:105DA000ACEEB4EFA50194010E94ED2DC60ED71EF6
:105DB000E81EF91EF7FE06C081E0C81AD108E10806
:105DC00080E8F80AC882D982EA82FB82C701B6015C
:105DD0009F77DF91CF91FF90EF90DF90CF90BF90B2
:105DE000AF909F908F9008950E94A82E089586E00E
:105DF00091E00E94A82E0895609306017093070118
:105E0000809308019093090108952F923F925F9229
:105E10006F927F928F929F92AF92BF92CF92DF92BA
:105E2000EF92FF920F931F93CF93DF938B01EA01C1
:105E30006115710521F0DB018C9311969C932097DD
:105E400039F09E01225031092332310508F0D8C0C3
:105E50007C016701BFEFCB1ADB0A5601F7016080B6
:105E6000862D90E00E943730892B11F07601F1CF1A
:105E7000FDE26F120AC0570182E0A80EB11CD701E3
:105E800011966C90772473940BC0BBE26B1207C021
:105E90005701E2E0AE0EB11CD70111966C90712C47
:105EA000CE018F7E892B89F4B0E36B1237C0F501E8
:105EB00080818F7D8835D1F46180F2E0AF0EB11C16
:105EC000872D8260782EC0E1D0E0CA30D10551F133
:105ED000C031D10521F0C830D10599F409C0CC24D6
:105EE000CA94DC2CEC2CAFE0FA2E22C0209769F784
:105EF000C8E0D0E0CC24CA94DC2CEC2CFFE1FF2ECF
:105F000017C06FEF7FEFCB019E01442737FD40950F
:105F1000542F0E94162E69017A010AC02097A9F613
:105F2000CAE0D0E0E9E9CE2EDC2CEC2CE9E1FE2E33
:105F3000F50160E020E030E0A9014E01AA2497FCC1
:105F4000A094BA2C1F0170ED572E560CA9E0A51590
:105F500070F48FEB860D8A3118F499EC592E06C037
:105F60008FE9860D8A3148F589EA582E560C852D21
:105F700090E08C179D070CF56F3FD9F0C216D30641
:105F8000E406F50698F0C501B4010E94F22D9B01CC
:105F9000AC01852D90E0A0E0B0E0280F391F4A1F2A
:105FA0005B1F281739074A075B0710F46FEF01C022
:105FB00061E03196D1016C90C5CF0115110551F00A
:105FC000662311F0319703C071FE04C03297D801E7
:105FD000ED93FC9370FE07C0509540953095219548
:105FE0003F4F4F4F5F4F67FF10C082E290E09093AA
:105FF0008D0680938C066FEF7FEF8FEF9FEF07C0CA
:1060000060E070E080E090E002C0B901CA01DF9179
:10601000CF911F910F91FF90EF90DF90CF90BF90A5
:10602000AF909F908F907F906F905F903F902F9058
:106030000895FC0188279927E89421912032E9F3FB
:10604000293010F02E30C8F32B3241F02D3239F4C4
:10605000689404C00E946B30820F911D21912053DF
:106060002A30C0F31EF4909581959F4F08959111A9
:1060700050C0803219F089508550D0F7089548EC0F
:1060800053E00E9444300895FA01A191B081009735
:1060900019F41097E1F0CD01DC01CD010D90002045
:1060A00011F4C00113C0FB012191222319F0201526
:1060B000D9F7F3CFFB012191201519F41E92119607
:1060C00006C02223C1F70D900020A1F7D001FA01EC
:1060D000A193B08308957AE0979F902D879F802D9C
:1060E000910D11240895F999FECF92BD81BDF89AC2
:1060F000992780B50895262FF999FECF1FBA92BD32
:1061000081BD20BD0FB6F894FA9AF99A0FBE019698
:0C6110000895992788270895F894FFCF80
:10611C0000008E06200001000000FF0002000200BB
:10612C000200020002000200020002000200020053
:10613C00020002000200020002000280250000059D
:10614C00400AA1204EA50020244EA52C2330C012BD
:10615C0000001A400AA1204EA5001B1E27522C231A
:10616C00308025000005400AA1204EA50020244EB9
:10617C00A52C2330004B000006400AD0009D49009E
:10618C007B289D492C233000E1000005400A450185
:10619C00D7DC03B81E0EBF00232E48E801008A404E
:1061AC000A6001555502AD1E20000023C801545849
:1061BC002074696D656F75742100596573004E6F9D
:1061CC00002C00386368004E2F41002C205B005DD2
:1061DC002028002900486F70206368616E6E656C22
:1061EC00200020402000456E746572696E67206146
:1061FC0064617074697665206368616E6E656C208D
:10620C0073656C656374696F6E2C207069636B6960
:10621C006E673A007363616E6E6572206D6F6465B4
:10622C00004E4F5420454E41424C45440053656E40
:10623C0064696E672073657474696E677320746F1C
:10624C002052580A00526573657474696E67207326
:10625C00657474696E6773206F6E2052580A004122
:10626C00626F727465642065646974730A00696E88
:10627C0076616C69642073656C656374696F6E001C
:10628C000D0A496E76616C696420696E70757420B4
:10629C002D20646973636172646564210700536522
:1062AC007474696E677320736176656420746F20F3
:1062BC00454550524F4D0A005265766572746564BF
:1062CC002073657474696E67732066726F6D2045F8
:1062DC004550524F4D0A004C6F61646564206661F5
:1062EC0063746F72792064656661756C74730A00EF
:1062FC004B657920616E64206368616E6E656C73AA
:10630C002072616E646F6D697A65640A004F706506
:10631C006E4C52536E6720545820737461727469BA
:10632C006E672000206F6E20485720006D6F6475DB
:10633C006C65206C6F636B65643F00342B340038E4
:10634C0000382B340031320031322B34003136001E
:10635C0050504D0052535349005344410053434C49
:10636C0000525844005458440041494E004C424598
:10637C0045500053504B54524D005342555300530B
:10638C00554D44004C4C494E440000070B0C101169
:10639C001500B7012B032F033103350338033D03DD
:1063AC00B7014003440349034D03510355035903FB
:1063BC005D0363036A036F0374038D028D028D0208
:1063CC008D02160A1322312900000000182C1D2AF8
:0863DC00BE2BEB2BD02B0D2C86
:107E00000F92CDB7DEB7112484B714BE81FFF1D035
:107E100082E08093C00088E18093C10086E0809377
:107E2000C20080E18093C4008EE0CDD088249924E4
:107E3000CC24C394F5E0DF2EE1E1EE2E73E0F72EC3
:107E4000B6D0082F813479F4B2D08983C2D0898129
:107E5000823811F481E005C0813811F485E001C059
:107E600083E09ED09AC0823411F484E103C085344B
:107E700019F485E0B6D091C0853561F498D0082F0B
:107E800010E095D090E0982E8824802A912A880CC2
:107E9000991C82C0863521F484E0A3D080E0E1CF34
:107EA000843609F04CC083D082D0A82E80D0B82E62
:107EB00000E011E07CD0F80181938F01AE16D1F77C
:107EC00088D0FB2DF53489F4E0E0F1E00BC0F9999E
:107ED000FECF92BC81BC0894811C911C819180BD15
:107EE000FA9AF99AEA1598F358C08B2D863409F05E
:107EF00054C0F401F7BEE89507B600FCFDCFF401CD
:107F0000A0E0B1E02C9130E011968C91119790E0B7
:107F1000982F8827822B932B12960C01C7BEE895C9
:107F20001124329681E0A038B80761F7F401D7BE7A
:107F3000E89507B600FCFDCFE7BEE8952EC0843774
:107F4000F1F435D034D0182F32D0B82E42D0FB2DDA
:107F5000F63421F4F40105914F010CC0FB2DF534EA
:107F600049F4F999FECF92BC81BC0894811C911C04
:107F7000F89A00B5802F14D0115049F70EC08537FC
:107F800039F427D08EE10CD085E90AD08FE069CF93
:107F9000813511F488E017D01CD080E101D050CF9A
:107FA0009091C00095FFFCCF8093C600089580910A
:107FB000C00087FFFCCF8091C00084FD01C0A89560
:107FC0008091C6000895E0E6F0E098E19083808318
:107FD0000895EDDF803219F088E0F5DFFFCF84E10E
:107FE000DFCF1F93182FE3DF1150E9F7F2DF1F9166
:0E7FF0000895282E80E0E7DFEE27FF27099492
:027FFE0001057B
:0400000300007E007B
:00000001FF
